:100000005F232130840084280B1D0900A400030E07
:10001000A3008312061D0E28A5011328250FA50095
:100020004120FF30B000061C1728A6011C28260F0F
:10003000A6004120FF30B000861D2028A7012328FC
:10004000270FA70041202E082F0403192C28AF0FDB
:100050002C28AE0F2C28B1152B08031DAB032C0A3E
:10006000031935282C08031DAC03300803193B285D
:10007000B00B3B283116230E8300A40E240E0B1167
:100080000900FC30AE001830AF000800820754347D
:100090005834003452345834003455344E3400341B
:1000A0004C344F3443344B344534443400342034DE
:1000B00020340034203444344934533450344C34E4
:1000C00041345934203400344D3455344C34543494
:1000D00000344D344134583400344D3449344E34B6
:1000E000203400342034563443344F3420344F34D9
:1000F00046344634533445345434203400342034A8
:100100004D3448347A3400344330A0008001840AEE
:10011000A00B862807309F008316303085002D30D5
:10012000860004308100831206171B22861DB1163B
:1001300083238101A0308B004120B111F021583080
:10014000E721E421E4218A30F1210930F721C03090
:10015000F121E6218021B1199C2893238030F121DF
:10016000861EB728311FB11731175230BB28311BFB
:10017000B11731135430E7218830F1210630311D99
:10018000C428331FC4281030F721B11FCA28B01B60
:10019000E228B113311FD72838304A2367233C3077
:1001A000582343233E30582336233830E1283A3051
:1001B0004A236723423058234323443058233623AD
:1001C0003A305123D0219321B11EAB28F6232D1CA8
:1001D000AB28EB211330F7211D30F721B1199C28F2
:1001E000D021C7232D18B70AD8232D18B703013003
:1001F00037020318FD280130B70015303702031C01
:1002000003291430B700D6013708D7000A30570247
:10021000031C0D29D700D60A06298E30F121560875
:10022000303EE7215708303EE721BE232D1CEE2843
:10023000F0212630F7210330F7211330F7218021F8
:10024000B1199C28D0213C3088213C305123932186
:10025000BE232D1C2029F0212230F721B1199C2822
:10026000D0213E304A2367233C3086213E30512343
:100270009321BE232D1C2E29F0210330F7212B3092
:10028000F721B1199C28D0214030BF2140305123A3
:100290009321BE232D1C4129F0212630F721003067
:1002A000F7211330F721B1199C28D0214230882141
:1002B000423051239321BE232D1C5329F02122309B
:1002C000F721B1199C28D02144304A2367234230BA
:1002D0008621443051239321BE232D1C6129F02116
:1002E0000030F7212B30F721B1199C28D02146305E
:1002F000BF21463051239321BE232D1C74299C28F5
:10030000CA30F1213830F721E521080058238C2923
:100310004A236723CD01CE0143235F30CD00503007
:10032000CE0036230800B1104B09C039031D9F29A8
:10033000B114CB09CC090130CC070318CB0A37081C
:10034000CA000310CA0DCA0DCA074A08CA00031022
:10035000CA0DCA0DCA074A08CA000310CA0DCA0D41
:10036000CA07FF22A722C130F1215530840009308D
:10037000A0000008E721840AA00BB92908004A233D
:100380008030CB0667238130CD009030CE003623FD
:100390007E30CD007030CE0043238030CB06080085
:1003A0005522861ED92938304A2335305123403012
:1003B000DE293A304A2335305123463058231F2353
:1003C000312235304A230800E621E6212030B500ED
:1003D000B6000517002A0130F1211830602308000B
:1003E0008130B500B6000513002205170800B400DF
:1003F0004620FF3903190800E7213408013EF72998
:100400008B13861383163030850083128517B60E42
:100410000F30B6050508F0393604850085138517B9
:100420000F30B5050508F0393504850085134B30CC
:10043000A3228B17080086012C222C222C2242306A
:10044000850085135F232830F1210830F121EB214D
:100450000630F1210C30F1295F23433085008513EC
:100460000800B21031157C230F30CD00A030CE0033
:1004700043235D30CD00C030CE00362348305823B2
:100480002D230319522A483051238822C2307A2260
:100490004B087A224C087A22AE307A22FF307A2238
:1004A0008D223313B21831110800331F5B2A2C0838
:1004B000031D6E2A77228822C3307A220830A000DA
:1004C000A2220616A222060C060CB30D0612A00BE1
:1004D000602A9E2294228D22331B7722861E331F90
:1004E000752A311D752A06130800061708006E309C
:1004F000AC000800B4000830A000B40D03189E2220
:10050000031C99229422A00B7D2A9E22942208008B
:1005100006169E22A2229922962A9922A222061625
:10052000A2229E22A2220800A2220616A2220612BF
:10053000080086108316861083120800831686141E
:10054000831208000F30A100A10BA42A0800031099
:100550001830A000D601D801DB01DD01D30DD20D8A
:10056000D10DDD0DDB0DD80DD60DA00BDA2A5D0EF9
:10057000DC005B0ED900580ED700560ED5003110A6
:100580005530EF225630EF225730EF225830EF220D
:100590005930EF2231145B30EF22A530DA005C30A5
:1005A000EF225D30EF22B11C0800540884002D308A
:1005B000800008005D30E3225B30E3225830E32204
:1005C0005630E322AE2A840003300007B400B41989
:1005D000800030300007B400B41B800008008400A5
:1005E0000F3000050319F82A303E8000311408004E
:1005F0003118F42A203080000408D4000800D30108
:100600004B08D1004C08D2000830A000CA0C0318D7
:100610000E2BA00B062BD101D20108000310192BC1
:10062000CA0C031C192B4C08D2074B0803184B0F9C
:10063000D107D10CD20CD30CA00B102B08004E0804
:10064000CC074D0803184D0FCB0708004E08CC020D
:100650004D08031C4D0FCB0208004E084C02B4009D
:100660004D08031C4D0A4B02340408004D08CF000E
:100670004E08D0000130CE070318CD0A2D23031CED
:1006800008004F30472B2D23031808004D304A2314
:10069000B214080084000008CB00840A0008CC00D3
:1006A000080084004B088000840A4C088000080081
:1006B00084000008CD00840A0008CE0008007630CF
:1006C000A100A201A20B622BA10B622B0800CD019D
:1006D0000130861D1430CE00CF232D181F23E023B8
:1006E0002D1826230230861DC830CE00C7232D18B2
:1006F0001F23D8232D1826234B09C039031D0800BA
:10070000CB01CC01080083169B0183123730840093
:100710001130A000AA23800083169B0A8312840A4A
:10072000A00B8A2B0800311E0800311283169B0192
:100730008312373084001130A000AA23000203196D
:10074000A32B0008AF2383169B0A8312840AA00BF5
:100750009D2B080083161C141A08831208008C13A2
:1007600083169A001C158B1355309D00AA309D00EE
:100770009C148B1783128C1FBB2B08001E30B400F7
:100780002A08AD002702E9232708AA0008006430E0
:100790002502031CCF2B4630A5006630D02B3C3001
:1007A000B4002808AD002502E9232508A8000800A8
:1007B00064302602031CE02B4630A6006630E12B95
:1007C0003C30B4002908AD002602E9232608A90020
:1007D00008000318F32B2D08053C0318F32B2D08F4
:1007E0003402FF30031C0301AD000800BE232D1CA2
:1007F00008002B080319FD2B08001930AB00F32B60
:02400E00783FF9
:1042000001004B0000004B0000004700E00054009C
:104210006000000000004700E00054006000000063
:0242200000009C
:00000001FF
